:020000040800F2
:1000000048200120A52C0008053000080530000814
:100010000530000805300008053000080000000029
:100020000000000000000000000000000530000893
:100030000530000800000000053000080530000809
:080040009C1300000100000008
:1000480010B50023934203D0CC5CC4540133F9E7C4
:0200580010BDD9
:10005A0002440346934202D003F8011BFAE77047B1
:10006A0010B5C9B20244904206D003461C7801304A
:0C007A008C42F8D1184610BD002010BDCB
:1000860038B504460D4600F028F82946204400F00D
:0600960018F8204638BDF9
:10009C0038B504460D4600F01DF82946421C204692
:0600AC00FFF7DDFF38BD87
:1000B20038B504460D4600F012F82946421C204687
:0600C20000F0EEF838BD6D
:1000C80038B5054608460C4600F006F82146421C9D
:0800D8002846FFF7B5FF38BD13
:0E00E0000023C25C0AB10133FBE718467047EB
:1000EE000023C25C1AB18B4201D00133F9E71846E6
:0200FE00704749
:1001000030B50023C45C3CB14A1E12F8015F1DB13A
:0C011000AC42FAD10133F5E7184630BDCF
:10011C0030B56FF0004485B00025CDE900454FF0B7
:10012C0000444FF0FF35CDE90245012302F0CEFD2E
:04013C0005B030BD1D
:100140001FB56FF000420023CDE9002300214FF0DE
:1001500000424FF0FF33CDE902230A220B4602F0A2
:08016000BBFD05B05DF804FBD6
:100168001FB56FF000420023CDE9002300214FF0B6
:1001780000424FF0FF33CDE902230A220B4602F07A
:08018800A7FD05B05DF804FBC2
:040190000020704794
:02019400FEE784
:10019600F8B5054608460E46FFF79FFF07462C466C
:1001A6002378013543B1204631463A4600F02FF810
:0C01B6000028F4D12046F8BD1846F8BD22
:1001C20030B50023C45C44B14A1E12F8015F15B178
:0E01D200AC42FAD101E00133F4E7184630BD2B
:1001E000F8B50546084616460F46FFF779FF013079
:1001F000B04234BF04463446394628462246FFF70B
:1002000023FFA64204D928190021321BFFF725FF3E
:040210002846F8BDC7
:1002140070B5154604460E46FFF760FF421C314692
:0E0224002046AA4228BF2A4600F039F870BDD5
:1002320038B50446CDB2FFF752FF231818460278AC
:10024200013BAA4203D0C4F10100C018F6D138BD67
:10025200F8B50E4604461746FFF741FF251830460B
:10026200FFF73DFFB84238BF0746314628463A46B7
:0C027200FFF7E9FE0023EB552046F8BD25
:10027E00884210B507D80023934203D0CC5CC454F7
:10028E000133F9E710BD12F1FF3202D38B5C8354B8
:04029E00F9E710BDAF
:1002A20030B50023934206D0C55CCC5C01332C1BD5
:0A02B200F8D0204630BD002030BD1A
:1002BC002DE9F04F0F468FB00021541C0D91127890
:1002CC00804610B117B1017000E0074600214FF0D5
:1002DC00FF390E460D468A468B46002A00F00882EE
:1002EC000629FDD8DFE801F0041834596090CA00E3
:1002FC00252A09D0DDF834C00CF10100B84238BF12
:10030C0008F80C200D9037E0002601214FF0FF3942
:10031C003546B246B3462FE02B2A13D007D8202AF5
:10032C0013D0232A40F0DC8145F0080524E02D2A67
:10033C0005D0302A40F0D48145F010051CE045F082
:10034C00010519E045F0020516E045F0040513E03F
:10035C00AA48805C400712D5303AD2B26FF0004008
:10036C00801A4FF00A0C90FBFCF0864202DD4FF035
:10037C00FF30D1E10CFB062622780134ADE72A2AA6
:10038C0040F0B0811E68191D002E2278BCBF45F0CC
:10039C00010576420B460134A4E12E2A40F0A481DB
:1003AC0022780421013498E79448B9F1FF3F10F802
:1003BC0002C008BF4FF000091CF0040F0DD0303AFA
:1003CC00D2B26FF00040801A4FF00A0C90FBFCF098
:1003DC008145CCDC0CFB0929CEE72A2A07D11A6807
:1003EC00013422EAE279043314F8012C7CE12D2A41
:1003FC0040F07A8114F8012B815C01F0040101F0CA
:10040C00FF090029F6D16FE16C2A23D00AD8682A9B
:10041C0012D06A2A40F06A812278062101344FF00A
:10042C00080A5AE7742A23D07A2A40F05F8122788E
:10043C004FF0060A013459E12278682A04D00134BD
:10044C0006214FF0020A48E76278062102344FF089
:10045C00010A42E722786C2A04D0013406214FF0BD
:10046C00030A3AE76278062102344FF0040A34E7B3
:10047C002278062101344FF0070A2EE76E2A00F08D
:10048C0009810DD8632A33D005D8582A40F01D8134
:10049C0045F040053AE1642A2CD0692A2AD014E1AF
:1004AC00732A00F093801DD86F2A43D0702A40F035
:1004BC000C811A6803F1040C0023CDE9002345F0EC
:1004CC008805102302930396CDF8109005954046AD
:1004DC000DA93A46CDF820C002F078FCDDF820C01A
:1004EC006346F9E0752A2AD0782A00F00F81ECE0F7
:1004FC000D995DE00AF1FF32072A13D8DFE802F00C
:10050C000407120A1212120A93F900000BE0B3F955
:10051C00000008E0073323F0070202F10803D2E9D8
:10052C00000102E01868C11704330A22CDE900016A
:10053C00029228E0BBF1000F00F0EB8004E0BBF16D
:10054C00000F01D14FF00A0B0AF1FF3245F0800584
:10055C00072A11D8DFE802F0040610081010100862
:10056C0018780AE0188808E0073323F0070202F134
:10057C000803D2E9000102E0186800210433CDE938
:10058C000001CDF808B00396CDF8109005954046C3
:10059C000DA93A46089302F019FC089B9CE0BA425C
:1005AC0004D208EB0201202001F8010C013E114697
:1005BC00012E01F10102F2DC181D1B68BA420D91EB
:1005CC0038BF08F801300D92034685E0181D0B90DA
:1005DC00B9F1FF3041421A684141099102B9084A08
:1005EC000023D15C31B9F31AE90723EAE3730CD584
:1005FC005B420AE0099828B10133F2E74C1200087B
:10060C00BC3F00084B45F7DBEDE70D9907910798C8
:10061C001844401A002809DD0131B942F7D208EB21
:10062C0001004FF0200C00F801CCF0E7079823EA0A
:10063C00E371013A5B1A01440A920D914A460A98F9
:10064C0010F8011F0A9089B1099848B1DDF834C03F
:10065C000CF10100B84238BF08F80C100D90EEE711
:10066C00002A02F1FF3001DD0246EFE70D991A4630
:10067C0062B1481CC01A1044B84205D2C81A404492
:10068C004FF0200C00F802C00132F1E7CB1A0D93A9
:10069C000B9B21E00AF1FF300D9A191D072810D889
:1006AC00DFE800F004070F0A0F0F0F0A1B681A701F
:1006BC0009E01B681A8006E018680023C0E90023D3
:1006CC0001E01B681A600B4606E00D98411CB9420C
:1006DC0038BF08F800200D91227800210134FCE588
:1006EC000221FAE50321F8E50521F6E50621F4E5FA
:1006FC000D98B84202D208F8002003E017B1474425
:10070C0007F8012C064B984206D930E64FF0100B37
:10071C001AE74FF0080B17E70FB0BDE8F08F00BFDA
:04072C00FEFFFF7F4E
:100730000CB407B504AB53F8042B0193FFF7BEFDCF
:0A07400003B05DF804EB02B070474F
:10074A0010B50C4613466FF000412246FFF7B1FD83
:02075A0010BDD0
:10075C000EB403B503AA52F8041B0192FFF7EFFF86
:0A076C0002B05DF804EB03B0704723
:0407760000207047A8
:10077C00024B5A6F42F080725A6770470038024041
:10078C00038819B19BB243F0010303E023F001038A
:08079C001B041B0C03807047D5
:0C081000014B01229A607047003002404A
:0C081C00014B1860186870470030024063
:1008280000EB81018842044B03D050F8042B1A6076
:0C083800F8E71868704700BF003002406D
:0C084400014B1868704700BF00300240F4
:10085000044B9A6809B1104301E022EA0000986055
:08086000704700BF002004E016
:10086800044B1A69002A04DA034A5A6002F18832F2
:0C0878005A607047003C024023016745B5
:10088400024B1A6942F000421A617047003C024070
:0C089400014BD860704700BF003C0240E0
:1008A0000B4BDA68D1030CD4DA68D2060BD4DA68C1
:1008B00012F0EF0F09D1DB689B074CBF072008201F
:1008C000704701207047052070470620704700BF21
:0408D000003C0240A6
:1008D40070B5064631B1012906D0022907D14FF47B
:1008E400007506E00D4604E04FF4807501E04FF416
:1008F400407500F0B9FB08281ED1104C236923F47D
:100904004073236123691D432561236923F0F803A0
:100914002361236943F002031E432661236943F4E0
:100924008033236100F0A0FB236923F002032361D9
:10093400236923F0F803236170BD00BF003C02402B
:1009440070B505460E4600F08FFB082811D1094CFE
:10095400236923F44073236123692361236943F0EA
:10096400010323612E7000F07FFB236923F0010350
:08097400236170BD003C02404C
:0C097C00014B1860704700BF00300040C5
:0C098800014B5860704700BF0030004079
:0C099400014B9860704700BF003000402D
:1009A000024B4AF6AA221A60704700BF003000408E
:1009B000024B4CF6CC421A60704700BF003000403A
:0C09C000014B1860704700BF20000E4281
:0C09CC00014B1860704700BFA0000E42F5
:1009D800034B5B6818420CBF00200120704700BF22
:0409E800007000405B
:1009EC00024B1A6842EA80001860704700700040A1
:1009FC000A4B00211A6842F001021A6099601A68C9
:100A0C0022F0847222F480321A60054A5A601A6805
:100A1C0022F480221A60D960704700BF003802406F
:040A2C001030002462
:100A3000064B002201281A701A7002D0042802D036
:100A400070471870704705221A707047703802405E
:100A50001D4B10B59A6802F00C02042A03D0082A34
:100A600003D01A4B18E01A4B16E059685A6811F473
:100A7000800F596814BF164B144B02F03F02B3FBB2
:100A8000F2F3114AC1F3881152684B43C2F3014299
:100A900001325200B3FBF2F30B4903608B680D4A3D
:100AA000C3F30313D45C0368E34043608C68C4F36E
:100AB0008224145D23FA04F484608968C1F342310E
:100AC000525CD340C36010BD003802400024F400E3
:080AD00040787D01C33F0008DE
:100AD80000F44073B3F5407F084B08D1996820F0C3
:100AE800704221F4F81122F440720A439A601A6F96
:100AF800C0F30B0010431867704700BF003802406E
:0C0B0800014B1860704700BF3C0E4742D4
:100B1400044B1A6B09B1104301E022EA0000186388
:080B2400704700BF00380240D9
:100B2C00044B1A6C09B1104301E022EA000018646E
:080B3C00704700BF00380240C1
:100B4400044B5A6C09B1104301E022EA00005864D6
:080B5400704700BF00380240A9
:100B5C00044B1A6909B1104301E022EA0000186144
:080B6C00704700BF0038024091
:100B7400044B5A6909B1104301E022EA00005861AC
:080B8400704700BF0038024079
:100B8C00044B9A6909B1104301E022EA0000986114
:080B9C00704700BF0038024061
:100BA400044B1A6A09B1104301E022EA00001862FA
:080BB400704700BF0038024049
:100BBC00044B5A6A09B1104301E022EA0000586262
:080BCC00704700BF0038024031
:100BD4004309012B074A01D1136803E0022B0CBF20
:100BE400136F536F00F01F0023FA00F000F00100B0
:080BF400704700BF0038024009
:100BFC00002382B001930D4BDA68520613D44FF0E8
:100C0C00FF32DA60094BDA68019902F040020131D7
:100C1C0001910199B1F5803F01D0002AF2D0D8683A
:100C2C00C0F3801000E0012002B0704700280040A3
:100C3C00024BDA6822F08002DA607047002800402C
:100C4C0038B50F4CCA236362532363620546FFF722
:100C5C00CFFF88B1A36823F04003A360A2682B6880
:100C6C001343A360AB68236123696A6843EA0243B8
:100C7C002361FFF7DDFF0120014BFF225A6238BDD3
:040C8C0000280040FC
:100C9000002382B001930E4BCA225A6253225A6239
:100CA000DA6822F0A002DA60094BDA68019902F0F2
:100CB0002002013101910199B1F5004F01D0002AC4
:100CC000F2D0D868FF22C0F340105A6202B07047D9
:040CD00000280040B8
:100CD400224A2DE9F0410B780C464F788E789268C1
:100CE40020B912F0400225D1CA7023E012F040026C
:100CF40000D1CA703F0247EA0343E5781E4346EA3F
:100D04000545164CCA23636253236362FFF774FFDD
:100D140058B105F07F3020F0FE402060FFF78CFFD3
:100D2400FFF7B4FF003018BF01200C4BFF225A62BA
:100D3400BDE8F081184600F012FA8046384600F00B
:100D44000EFA0746304600F00AFAE57840EA054014
:100D540040EA084545EA0725D3E700BF00280040DC
:100D64000F4B70B51B680C46C3F30542C3F306264C
:100D740003F07F0503F480031B0C0A704E708D7022
:100D8400CB7058B9104600F0F7F92070304600F0E7
:100D9400F3F96070284600F0EFF9A07070BD00BF51
:040DA40000280040E3
:100DA8002DE9F0410C464B78CA788F780E7878BBDD
:100DB800D90603D523F010030A336370104600F0F8
:100DC800CCF98046607800F0C8F90446384600F04F
:100DD800C4F940EA463040EA084545EA0425104C83
:100DE800CA23636253236362FFF704FF58B125F0F7
:100DF8007F4323F0C0036360FFF71CFFFFF744FF46
:100E0800003018BF0120064BFF225A62BDE8F0816E
:100E18001D0245EA02453D4345EA4635DFE700BF86
:040E2800002800405E
:100E2C000E4B70B55B680C46C3F30742C3F3042644
:100E3C0003F03F05C3F34233CA704E708D700B70D4
:100E4C0058B9104600F094F9E070304600F090F973
:100E5C006070284600F08CF9A07070BD002800402E
:100E6C00084B9A6822F4006222F0080209B142F49D
:100E7C0000621043CA225A6253225A62FF229860BF
:080E8C005A6270470028004083
:100E940082B000230193054B0193019B03EB800077
:100EA4000190019B196002B0704700BF50280040B8
:100EB40082B000230193054B0193019B03EB800057
:100EC4000190019B186802B0704700BF5028004091
:100ED400044B1A6C22F400321A641A6C104318641E
:080EE400704700BF0028004028
:100EEC000D4BCA225A6253225A6220F0040200F0BF
:100EFC00040029B199680A439A601A6C104306E001
:100F0C00996821EA02029A601A6C22EA00001864BD
:0C0F1C00014BFF225A6270470028004081
:100F2800054BDB6823F088039B049B0C03420CBF32
:0C0F380000200120704700BF002800408E
:100F4400054B80B2DA6840F0800002F0800262EA69
:0C0F54000002DA60704700BF0028004077
:100F600008B5134B98420AD14FF480500121FFF786
:100F700025FE4FF480500021FFF720FE08BD0D4BE9
:100F8000984207D14FF480400121FFF70BFE4FF448
:100F9000804009E0084B984209D14FF400400121FC
:100FA000FFF700FE4FF400400021FFF7FBFD08BDF6
:0C0FB0000030014000380040003C0040D0
:100FBC00038ACA889BB223F4405330B513430D46C1
:100FCC0003820989AB8882890B43698992B20B43EE
:100FDC0022F4B05222F00C029BB213438381838A19
:100FEC00AA899BB223F44073134385B083820446D1
:100FFC006846FFF727FD194B9C4203D003F580632D
:10100C009C4201D1039B00E0029BA289192112B2E0
:10101C005943002A2A684FF06403B4BF520092006F
:10102C00B1FBF2F1B1FBF3F21201100903FB101149
:10103C00A08900B2002806DAC9003231B1FBF3F303
:10104C0003F0070305E009013231B1FBF3F303F0C0
:10105C000F031A4392B2228105B030BD001001403B
:10106C0007B508238DF80730FFF714FC8DF807003F
:10107C009DF80730012BF7D09DF8070003B05DF801
:02108C0004FB63
:10108E002DE9F0410F68002301229A4002EA07057C
:10109E00954230D15A00032494400668E44326401A
:1010AE0006600E79D0F800C006FA02F8013E48EA52
:1010BE000C0C012EC0F800C014D891F805C086683B
:1010CE000CFA02FC2640866086684CEA06068660AC
:1010DE00466826EA050545608D7946689D40ADB2A5
:1010EE0035434560C5682C40CD79C46005FA02F2DF
:1010FE00C4682243C2600133102BC5D1BDE8F08114
:10110E004FF6FF7303600023037143718371C37144
:02111E00704718
:0C112000036919420CBF00200120704739
:04112C000183704784
:041130004183704740
:0A1134000AB1018370474183704740
:10113E0001F00703C90800EB81009B000F219940C5
:10114E009A4010B5046A24EA01010162016A114352
:04115E00016210BD5D
:1011620000230928DAB203F1010302D90A38C0B216
:0A117200F7E740EA0210C0B2704730
:10117C00030903EB830300F00F0000EB4300C0B244
:02118C007047AA
:0C118E0000217F22FF2380E80E00704744
:0C119A000023C370037043708370704723
:0E11A60001230370837043700023C3707047F1
:1011B4000B8810B54C88028823438C8802F4415272
:1011C4002343CC8823430C8923434C8923438C89B0
:1011D4002343CC89234313439BB20380838B23F49F
:0E11E40000631B041B0C83830B8A038210BD67
:1011F200038819B19BB243F0400303E023F040039C
:081202001B041B0C0380704764
:06120A00808980B27047EC
:041210008181704721
:0C121400038919420CBF00200120704724
:10122000838919B19BB243F4005303E023F40053C4
:081230001B041B0C83817047B5
:08123800C1F308018180704739
:0C124000038819420CBF002001207047F9
:10124C00202020202020202020282828282820206A
:10125C002020202020202020202020202020202082
:10126C00481010101010101010101010101010103A
:10127C0004040404040404040404101010101010DA
:10128C001081818181818101010101010101010133
:10129C0001010101010101010101011010101010E7
:1012AC001082828282828202020202020202020204
:1012BC0002020202020202020202021010101020AC
:1012CC000000000000000000000000000000000012
:1012DC000000000000000000000000000000000002
:1012EC0000000000000000000000000000000000F2
:1012FC0000000000000000000000000000000000E2
:10130C0000000000000000000000000000000000D1
:10131C0000000000000000000000000000000000C1
:10132C0000000000000000000000000000000000B1
:10133C0000000000000000000000000000000000A1
:10134C004BB942B9002908BF002802D04FF0FF3139
:10135C00084600F03BB882B0EC462DE9005000F096
:10136C001DF8DDF804E002B00CBC70472DE9704F9D
:10137C00089E14461D468046894600F029F804FB59
:10138C0001F3A4FB00AB00FB05329344B8EB0A0855
:10139C0069EB0B09C6E90089BDE8708F2DE9704F28
:1013AC00089E14461D468046894600F061F900FBF4
:1013BC0005F5A0FB04AB04FB0154A344B8EB0A08ED
:1013CC0069EB0B09C6E90089BDE8708F704700BF57
:1013DC0000292DE9F00FC0F2A1800024002BC0F2EF
:1013EC009880154606460F46002B3FD18A4258D9A5
:1013FC00B2FA82F34BB1C3F1200201FA03F720FADF
:10140C0002F29D4000FA03F61743290CB7FBF1F2E8
:10141C0001FB1277A8B200FB02F34FEA164C4CEA20
:10142C000747BB4209D97F1902F1FF3C80F00581C7
:10143C00BB4240F20281023A2F44FF1AB7FBF1F390
:10144C0001FB137100FB03F0B6B246EA014188427E
:10145C0008D9491903F1FF3780F0F180884240F236
:10146C00EE80023B43EA0242002303E08B420AD99E
:10147C0000231A461046194614B1404261EB410153
:10148C00BDE8F00F7047B3FA83F8B8F1000F40F0E5
:10149C0088808B4202D3824200F2E2800023012238
:1014AC00E8E712B90123B3FBF2F5B5FA85F2002A8D
:1014BC003AD17F1B280C1FFA85FC0123B7FBF0F1F6
:1014CC0000FB11770CFB01F24FEA164848EA07477C
:1014DC00BA4207D97F1901F1FF3802D2BA4200F2A1
:1014EC00C4804146BF1AB7FBF0F200FB12700CFB34
:1014FC0002FCB6B246EA0040844507D9401902F115
:10150C00FF3702D2844500F2AE803A4642EA0142ED
:10151C00B0E7E443524263EB430362E7404261EBC2
:10152C0041014FF0FF3459E79540C2F1200927FAE9
:10153C0009F126FA09F99740280CB1FBF0F800FBE9
:10154C0018111FFA85FC0CFB08F349EA07094FEA4E
:10155C00194747EA01418B4206FA02F608D94919A4
:10156C0008F1FF327AD28B4278D9A8F102082944CB
:10157C00C91AB1FBF0F300FB13170CFB03F21FFAB3
:10158C0089F949EA0747BA4207D97F1903F1FF31B4
:10159C0060D2BA425ED9023B2F44BF1A43EA0843D9
:1015AC008CE7C8F1200225FA02F103FA08FC27FAAD
:1015BC0002F320FA02F207FA08F741EA0C0C4FEAA0
:1015CC001C49B3FBF9F109FB11331FFA8CFA0AFB26
:1015DC0001FB17433A0C42EA03439B4505FA08F01A
:1015EC0008D913EB0C0301F1FF3235D29B4533D9EB
:1015FC0002396344CBEB0303B3FBF9F209FB12335F
:10160C000AFB02FABFB247EA0347BA4508D917EBFF
:10161C000C0702F1FF331BD2BA4519D9023A6744C1
:10162C0042EA0145A5FB0001CAEB07078F424FF0C8
:10163C0000030AD305D02A461CE76246FDE63B466A
:10164C0010E706FA08F68642F5D26A1E002311E767
:10165C001A46E5E70B46A0E71146CBE7904687E72D
:10166C004346424606E7023A50E702392F4439E72F
:10167C002DE9F00F144605460E46002B43D18A4245
:10168C0053D9B2FA82F757B1C7F1200620FA06F601
:10169C0001FA07F302FA07F400FA07F51E43210CCE
:1016AC00B6FBF1F201FB1266A0B200FB02F32F0CA9
:1016BC0047EA0646B34209D9361902F1FF3780F0E2
:1016CC00FD80B34240F2FA80023A2644F61AB6FB89
:1016DC00F1F301FB136100FB03F0ADB245EA0141EC
:1016EC00884208D9091903F1FF3680F0E980884255
:1016FC0040F2E680023B43EA0242002310461946C0
:10170C00BDE8F00F70478B424CD8B3FA83F6002E2D
:10171C004FD18B4202D3824200F2DD80BDE8F00F44
:10172C000023012210461946704712B90124B4FB5C
:10173C00F2F4B4FA84F2002A40F08280091B260CE1
:10174C00A7B20123B1FBF6F006FB101107FB00F268
:10175C004FEA154C4CEA01418A4207D9091900F1AC
:10176C00FF3C02D28A4200F2C8806046891AB1FB63
:10177C00F6F206FB121107FB02F7ADB245EA014582
:10178C00AF4208D92C1902F1FF3180F09B80A7429F
:10179C0040F29880023A42EA004210461946BDE8EF
:1017AC00F00F704700231A4610461946BDE8F00F9B
:1017BC007047C6F1200522FA05F703FA06F421FA60
:1017CC0005F301FA06FB20FA05F53C434FEA1448F1
:1017DC00B3FBF8FC08FB1C331FFA84F909FB0CFA69
:1017EC0045EA0B0B4FEA1B4545EA03439A4502FABF
:1017FC0006F204D91B190CF1FF356FD3AC46CAEBBA
:10180C000303B3FBF8F508FB153309FB05F91FFAC5
:10181C008BFB4BEA0347B94504D93F1905F1FF335C
:10182C0062D31D4645EA0C4CACFB0223C9EB0707FF
:10183C009F424FF000054AD346D062462B465DE7E7
:10184C009440C2F1200921FA09FC914020FA09F9CF
:10185C00260CBCFBF6F806FB18CCA7B207FB08F36A
:10186C0049EA01094FEA194141EA0C4C634500FA77
:10187C0002F509D91CEB040C08F1FF323BD263458D
:10188C0039D9A8F10208A444C3EB0C0CBCFBF6F349
:10189C0006FB13C107FB03F21FFA89F949EA014160
:1018AC008A4207D9091903F1FF3022D28A4220D982
:1018BC00023B2144891A43EA084343E73A4605E7C9
:1018CC00334618E70A4666E7B0409042B5D20CF1B1
:1018DC00FF32002312E7334632460FE79A458DD983
:1018EC00ACF1020C23448AE7B9459AD9023D27444E
:1018FC0098E70346DEE79046C6E70238214435E711
:10190C0010B5044608484021FFF794FC0028F9D094
:10191C0005482146FFF78AFC03484021FFF78AFC63
:10192C000028F9D010BD00BF00480040014608B5A2
:10193C000448FFF767FC03480221FFF765FC002809
:10194C00F9D008BD0038004000B9074803680133DE
:10195C0008D04368013305D0C069044BC31A584200
:10196C005841704700207047004000086F57654E83
:10197C00074B1A69C2F306427F2A07D11869C0F3D4
:10198C000C00B0F1FF0358425841704700207047DB
:10199C000028004000F13F4000F57E00800A082836
:1019AC000FD8084A52F820305BB1013B42F8203086
:1019BC003BB9012101FA00F0034B1A6B22EA00003B
:1019CC0018637047200000200038024000F13F40AF
:1019DC0000F57E00800A08280DD8074A52F82030FE
:1019EC00591C42F8201033B9012101FA00F0034BC5
:1019FC001A6B104318637047200000200038024017
:101A0C0010B50C4C2046FFF7E1FF072001F036FB28
:101A1C004FF4805100222046FFF786FB042001F092
:101A2C002DFB2046FFF7B6FF4FF480400021FFF757
:101A3C0077F810BD0004024010B50B4C01214FF497
:101A4C008040FFF76DF82046FFF7C0FF20464FF4AB
:101A5C0080510122FFF768FB072001F00FFB2046A5
:101A6C00FFF798FF10BD00BF0004024008B5FFF758
:101A7C00E3FF0020FFF75AFF0020FFF757FF00207D
:101A8C00FFF754FFFFF7BCFFFEF772FEBFF34F8F5B
:101A9C00044A054BD16801F4E0610B43D360BFF3FA
:101AAC004F8FFEE700ED00E00400FA05F0B55E256F
:101ABC006843204BB0FBF1F51A68ADF6DC3D95425E
:101ACC0034D002AC00214FF43D6220461D60FEF77D
:101ADC00BEFA1B238DE818001748102140226923F9
:101AEC0001F0AFFA08238DE8180014486023182180
:101AFC006A2201F0A6FA0DF2FA760DF28E7300222C
:101B0C00AA420DD002F11900C0B2C108012700F0A1
:101B1C00070007FA00F05F5C013238435854EFE7D6
:101B2C001233B342EBD1204601F0E3FA0DF6DC3D63
:101B3C00F0BD00BF08000020B03500084439000893
:101B4C002DE9F043ADF6DC3D02AC00214FF43D62D3
:101B5C0080462046FEF77BFA2C238DE818002022C5
:101B6C00284818215C2301F06CFA1C2215460F271B
:101B7C00974007EA0807D740234B242101FB07377E
:101B8C000DF50366002117F801C00023082B07D0C0
:101B9C000120984010EA0C0F0CBF0020012003E03C
:101BAC007818407800F0010078B15819C0B24FEAAB
:101BBC00D00E4FF0010900F0070009FA00F016F8FA
:101BCC000E9040EA090006F80E000133092BDDD116
:101BDC000231242906F11206D5D10B35742DA2F150
:101BEC000402C4D10E238DE81800102190226D231D
:101BFC00064801F026FA204601F07BFA0DF6DC3D92
:101C0C00BDE8F083A0330008A4390008DC320008DA
:101C1C0010B5ADF6D83D02AC204600214FF43D6224
:101C2C00FEF715FA1B238DE81800102140226923BA
:101C3C00044801F006FA204601F05BFA0DF6D83D97
:101C4C0010BD00BFB03500082DE9F74F434E444F8F
:101C5C0001214FF48040FEF763FF3046FFF7B6FEDC
:101C6C003846404CFFF7B2FE30460D210522FFF7F7
:101C7C0060FA052230460F21FFF75BFA3046214609
:101C8C000125FFF7FEF920233846214623602571F4
:101C9C00A5714FF0000A01934FF4805BFFF7F1F947
:101CAC00304621464FF002084FF48049257184F8E4
:101CBC0006A0C4F800B0FFF7E4F93046214684F8DA
:101CCC000480C4F80080FFF7DCF921462571A5716A
:101CDC00C4F80090244C3046FFF7D3F92046FFF7A8
:101CEC0039F920462149FFF75FFA20462946FFF7CC
:101CFC007AFA019B384619465246FFF715FA2A46DE
:101D0C0030464946FFF710FA40462946FEF708FFD1
:101D1C00A4F5505480232380F92323854FF4F042FB
:101D2C004FF6FF13E3623046A283294623644246F2
:101D3C00A4F820B0FFF7FDF929462046A582FEF74E
:101D4C001FFD3846FFF726FE3046FFF723FE4846B8
:101D5C005146FEF7E5FE03B0BDE8F08F00040240EB
:101D6C000008024000000020003800400C00002059
:101D7C0010B5074C2046FFF729FE20461021FFF72F
:101D8C00CFF92046FFF706FE012001F077F910BDD0
:101D9C000000024038B50A4B0C2404FB0034606888
:101DAC00FFF714FE21896068FFF7B4F905466068F7
:101DBC00FFF7F0FDD5F1010038BF002038BD00BFA2
:101DCC009432000810B5064C2046FFF7FFFD204664
:101DDC001021FFF7A7F92046FFF7DCFD10BD00BF6F
:101DEC0000000240F0B587B0FFF7C2FD002841D1DA
:101DFC000320FFF759F807460420FFF755F8474B27
:101E0C000A241A68C2F30545C2F30626C2F302136C
:101E1C0002F00F0204FB0322330906F00F0604FB49
:101E2C0003662B0905F00F0504FB03533C2505FB4A
:101E3C00036305FB0323191A44BF01F5A83101F50F
:101E4C00C07107EB91210320FFF71EF803A8FFF7E1
:101E5C0098F903A8FEF7F4FE01A8FFF798F901A979
:101E6C000020FEF731FF02A8FFF797F9002002A926
:101E7C00FEF794FF0A2442F2107501F05CF910B9D8
:101E8C00013DFAD107E0264D01F055F908B1013DAD
:101E9C00FAD1013CEFD10020FEF792FD00214FF268
:101EAC000400FFF71DF84FF43C50FFF745F81D4BAD
:101EBC0001201A6842F004021A60FEF781FD1A4BE9
:101ECC001B781BB1194801F055F908E01848FEF7CA
:101EDC0001F9174902461748FEF7DDF970B11648AB
:101EEC0001F048F90020FEF7EFFF08200121FEF772
:101EFC00B7FF4FF400400121FEF7F2FF0F4801F04D
:101F0C0039F9084B1A6842F002021A600C4B1A6934
:101F1C0042F004021A6130BF07B0F0BD0028004047
:101F2C00A086010000700040017AFF1F2A370008CC
:101F3C003F3700082078FF1F443700085937000846
:101F4C0000ED00E0B0F1006F10B504460BD20D4867
:101F5C0001F007F9204601F013F90B4801F00AF9DA
:101F6C004FF0FF3010BD094A002352F8041FA14264
:101F7C0002D851688C4202D30133072BF5D1184695
:101F8C0010BD00BF6D3800086A37000870320008B9
:101F9C0008B5024801F0EEF800BEFEE783370008F2
:101FAC0010B504460A480221FFF72EF90028F9D093
:101FBC0007482146FFF726F905480121FFF724F9C8
:101FCC000028F9D00248FFF71AF9C0B210BD00BFC3
:101FDC00003001402DE9F04F87B00121814600AF60
:101FEC000020FFF763FD042001F063F807F10C00FB
:101FFC0049460C2201F0E9F8FD683C690C2DD7F834
:10200C0014B013D0994801F0ACF8284601F0B8F898
:10201C00974801F0A6F8204601F0B2F8954801F077
:10202C00A0F8584601F0ACF8934833E0934801F01F
:10203C00A1F84FF480500121FEF766FD09F10C095F
:10204C00EA46FEF7DFFBA0B06E462546C846802D5B
:10205C000CD941463046802201F0B7F83046202199
:10206C00FEF7DCFB803D08F18008F0E725B1304637
:10207C0041462A4601F0A9F82946304600F0C6FF31
:10208C00002180464FF48050FEF73EFDD845D546E2
:10209C0004D07B4801F06EF80120E3E088B068467C
:1020AC004946202201F091F86846FFF74DFC786014
:1020BC007448D54601F05EF87B682BB9724801F084
:1020CC0059F804F5404600E02646002E3BD06F48F8
:1020DC00FFF738FF05466E483044FFF733FF002DFD
:1020EC00824630DB00282EDB431B01334FEA430BC7
:1020FC0000205946FFF7DAFCFEF7B0FB654B0026D3
:10210C0003EB45033B6055451BDCF320FEF7BCFBA2
:10211C003B68002133F81600FEF7D6FB082806F1C1
:10212C00010608D05C4801F01CF8284601F028F89C
:10213C0001F00FF805E030465946FFF7B7FC0135C2
:10214C00E1E7FEF799FB554801F014F87B680BB1F9
:10215C004E4B00E0524B7B6063083B600025A54270
:10216C003CD2661BB6F5803F28BF4FF480362EB1AB
:10217C004C4805EB0901324601F027F8D7F804A0CA
:10218C00FEF76CFBF320FEF77FFBAA444FF0000B2D
:10219C00B34519D043490BEB0A0011F80B10FEF7AD
:1021AC00CBFB08280DD0404800F0DBFF504600F078
:1021BC00E7FF00F0CEFFFEF75FFB3C4800F0DAFFD4
:1021CC000CE00BF1010BE3E7FEF756FB3B682146F5
:1021DC0003EB5500FFF76AFC5D44C0E7344800F0A0
:1021EC00C0FF204600F0CCFF324800F0C3FF0020B7
:1021FC00FFF7AAFB20B1304800F0BCFF234D03E0F1
:10220C002E4800F0B7FF264D4FF480500121A60850
:10221C00FEF77AFCFEF7F6FA31462846FEF7FEFA90
:10222C0004F0030105EB860000F0F0FE00210446EB
:10223C004FF48050FEF768FC214800F092FF4046B6
:10224C0000F09EFF1F4800F08CFF204600F098FF26
:10225C0000F07FFF444504D01B4800F08BFF0220A8
:10226C0000E000201C37BD46BDE8F08F8E3700081B
:10227C0097370008A1370008A8370008C7370008AF
:10228C00E4370008073800081A3800080040000836
:10229C00FF3F0008CC320008323800084A380008EA
:1022AC0000000108440000205D3800087638000862
:1022BC00813800088F38000896380008BB380008B1
:1022CC00E0380008F3380008F938000870B54FF40E
:1022DC0080500121FEF730FCFFF774FD0520164CF1
:1022EC00FFF75EFE002C04F1FF341FDCFFF740FD0E
:1022FC00FFF768FD9F20FFF753FEA920FFF750FE64
:10230C000546A920FFF74CFE0646A920FFF748FE1C
:10231C003602044646EA0545FFF72AFD4FF4805085
:10232C000021FEF709FC45EA040070BDA920FFF767
:10233C0037FEC307D6D4D9E70090D00308B50446BE
:10234C00114800F00EFF204600F01AFF00F001FFCC
:10235C002046FFF7F5FB00F0EEFE0C4B20F00400DE
:10236C0018701D4600F0E7FE2B7800F0FB0083424E
:10237C0001D10B2401E0FFF779FB013CF2D04FF4C3
:10238C007A7000F07BFEF8E7E43B00084400012083
:10239C0080B5464B4FF4C06290B01A6001214FF0EB
:1023AC008050FEF7BDFB0120FEF704FB4048FFF711
:1023BC000DFB4FF480200121FEF7B2FB3C480A21B3
:1023CC000722FEF7B6FE072239480B21FEF7B1FEB5
:1023DC0010AF4FF4806347F8383D00244FF00108EC
:1023EC000225334839468DF80E408DF80F808DF854
:1023FC000C508DF80D50FEF744FE4FF400632C4842
:10240C00394602938DF80C5004AEFEF73AFE4FF4A9
:10241C006133049327480C233146ADF81A30ADF8DC
:10242C001440ADF81640ADF81840ADF81C40FEF75E
:10243C00BFFD41461F48FEF7EDFE1D48FFF7AAFA07
:10244C001D4800F08EFE1D4B586F00F099FE00F0F9
:10245C0080FE7920FEF7B8FB404502D1184800F009
:10246C0089FE012000F010FE10B90121FEF70CFDD1
:10247C004120FEF7A9FB58BB124800F07BFE01205F
:10248C00FEF7D0FA47F230544120FEF79DFBF8B925
:10249C004FF47A7000F0F2FD013CF5D10A4800F0DF
:1024AC0069FEFFF7D1FB094837E100BF003C024051
:1024BC000008024000480040F03B00080038024091
:1024CC00003C0008103C0008283C0008114550FE58
:1024DC004FF48070FEF7FAFA0120FEF70FFBFEF7BF
:1024EC00D1FB0020FEF76CFA01214FF48040FEF77F
:1024FC0023FBBB48FFF76AFA3046FEF702FE0024C6
:10250C000125B74831468DF815408DF816408DF8E9
:10251C00174004958DF81450FEF7B3FD2246B048D1
:10252C002946FEF701FEAE48FFF734FAAD4C04F134
:10253C00300954F8040CFFF749FA3046FEF7E1FD78
:10254C00236854F8040C4FF000083146022504931C
:10255C008DF814808DF815508DF817800C34FEF71B
:10256C0090FD54F8100CFFF715FA4C45E1D14FF4DF
:10257C0080404146FEF7E0FA4FF4807000F084FD95
:10258C00002800F0CC804FF4807000F087FDFFF73E
:10259C0029FC954800F0EEFD0220FEF785FC9349DE
:1025AC00884202D00220FEF76FFC914800F0D9FD62
:1025BC000220FEF779FC00F0E3FD00F0CAFD4FF4B9
:1025CC00804000F061FD90B18A4800F0D3FD4FF4DB
:1025DC00804000F063FD082000F060FD102000F04A
:1025EC005DFD202000F05AFD402000F057FDFFF764
:1025FC002BFBFFF70DFB01214FF48050FEF79CFAEB
:10260C007748FFF7E3F901200146FEF77DFA052133
:10261C000A467348FEF78DFD714806210522FEF728
:10262C0088FD05226E480721FEF783FD0024022554
:10263C00C0236B4839468DF80C508DF80D50029321
:10264C008DF80E408DF80F40FEF71BFD20236448DB
:10265C0039468DF80F5002930125FEF712FD102319
:10266C0039465F4802938DF80C508DF80F50FEF7E9
:10267C0008FD6148FEF76EFC4FF48273ADF8123022
:10268C004FF40073ADF81A305B4807233146ADF8B0
:10269C002030ADF81040ADF81440ADF81640ADF850
:1026AC001840ADF81C40ADF81E40FEF77DFD2946E4
:1026BC005148FEF798FD4A48FFF76CF9FFF782FB8B
:1026CC00AB20FFF76DFCFFF753FB642000F0D6FC4A
:1026DC0021464FF48050FEF72FFAFFF7F7FD2846FE
:1026EC00FEF7E2FB25460490E8B2FFF753FB98BBDC
:1026FC0070550135042DF7D1049D3DB13F4800F0D4
:10270C0030FD284600F03CFD00F023FD0120294659
:10271C00FEF7BAFB002C3DD03948FFF70FFE2846D8
:10272C00FEF754F9012814D12846FEF759F94FF455
:10273C000060FEF7F3FB18B1324800F01BFDB9E066
:10274C00314C00F0F8FC002800F00481013CF8D179
:10275C00B0E000F0B9FC1CE7735D042B0ADD2B48DC
:10276C0000F008FD049800F00BFD01200021FEF79D
:10277C008BFB0FE00133DBB2042B7355B9DD24481E
:10278C0000F0EFFC284600F0FBFC224800F0F2FCC5
:10279C000124AEE7FFF79AFD1F4B0344012B01D92F
:1027AC001E48BAE71E4800F0DCFC0020FEF77CFB5C
:1027BC0000F0E6FC00F0CDFC802000F065FC18B1C8
:1027CC00802000F06BFC73E04FF4003000F05CFCF8
:1027DC00044638B34FF4003000F060FC04E100BF55
:1027EC00000002409C320008603C00087086415694
:1027FC009C3C0008B13C0008003001401F3D000823
:10280C00014550FE453C0008A0860100DE3C000856
:10281C000A3D0008153D0008EA44DFFF024550FE62
:10282C004B3D00080120FFF7B5FAD8B12046FFF761
:10283C00B1FAB8B1B74800F09DFC41F288340120E0
:10284C00FFF7A8FA002800F08B800020FFF7A2FA0F
:10285C00002800F085804FF47A7000F00FFC013CEA
:10286C00EDD1C1E00020FFF76FF808B1AA4B00E0F2
:10287C00AA4B0CCB013301D0013271D1A84800F026
:10288C0079FCB1E0A74800F075FC082000F006FCCC
:10289C00102000F003FC202000F000FC402000F091
:1028AC00FDFB0024042000F0F9FB002C40F0088113
:1028BC009D4832E7FFF75CF8002847D0002001A9BB
:1028CC009A4DFEF749FA344600203946FEF7A8FA2D
:1028DC000FCD0FC40FCD0FC495E80F0084E80F0087
:1028EC009DF8092010A901EB82039DF80BE053F829
:1028FC00343C40F26D1101FB0E3303EB9E030EF1E1
:10290C00010E1EF0030F02D1022A88BF01339DF87D
:10291C000A409DF80410013C2344182404FB0314C2
:10292C009DF805103C2202FB04149DF806100320B0
:10293C0002FB0414FEF7B8FA01190320FEF7A4FAFF
:10294C0004200021FEF7A0FA00F0BEFB784800F04E
:10295C0011FC1EE6774800F00DFCFFF743FAF5E793
:10296C007D20FEF731F970B94FF4007000F08CFB4C
:10297C0048B9714800F0FEFB082000F08FFB1020D6
:10298C0000F08CFB85E07D20FEF71EF910B16B4842
:10299C0000F0F0FB4FF4007000F076FB10B16848CB
:1029AC0000F0E8FB4FF4007000F078FB102000F012
:1029BC006BFB48B1634800F0DDFB082000F06EFBB8
:1029CC00102000F06BFB12E0082000F05DFB20B142
:1029DC005D4800F0CFFB102003E05C4800F0CAFB20
:1029EC00082000F066FB54E0594800F0C3FB59483E
:1029FC0000F0C0FB4FF40010FFF7ECFA10B1022806
:102A0C0028D809E0202000F049FB402000F046FBCC
:102A1C00802000F04EFB1DE0082000F04AFB102047
:102A2C0000F047FB202000F02FFB20B94A4800F0B3
:102A3C00A1FB202009E0402000F026FB00287FF4B9
:102A4C0021AF464800F096FB402000F032FB4FF4DB
:102A5C0000701AE0012425E7414800F08BFB0820A8
:102A6C0000F01CFB102000F019FB202000F016FBDE
:102A7C00402000F013FB2046FFF7ACFA022840F090
:102A8C00F080082000F015FB102000F012FBFEF780
:102A9C00EDFF022000F0F8FA90B1042000F0F4FAF7
:102AAC0004460028D8D02F4800F064FB042000F026
:102ABC00F5FA022000F0F2FA4FF4004000F0EEFAC2
:102ACC004FF4005000F0E0FA04464FF4805000F050
:102ADC00DBFA400040EA84044FF4006000F0D4FAC2
:102AEC00E4B22043431C03F0FF03013B4FF40060AE
:102AFC00062B58D8DFE803F03C383C043C383C004B
:102B0C0000F0CCFA4FF4805000F0C8FA4FF40050AB
:102B1C002EE000BF573D00080040000800000108EF
:102B2C00893D0008B33E0008034550FE44320008BE
:102B3C00503C0008523F00089C3D0008AD3D000889
:102B4C00C53D0008E53D0008FB3D0008113E0008AE
:102B5C00673F0008273E0008413E00087A3E000807
:102B6C00233F0008ED3E000800F098FA4FF4805027
:102B7C0000F09FFA45F25550FDF7FAFE0420FDF7E0
:102B8C00FDFE40F6FF70FDF7FFFE0020FDF7F0FEA6
:102B9C004FF480500121FDF755FE0020FEF7D4FEC6
:102BAC0068B9354B0CE000F079FA4FF4805000F026
:102BBC0075FA4FF4005000F071FA3048ADE5304B27
:102BCC005D6830481E6800F0CCFA284600F0D8FA50
:102BDC0000F0BFFA00F0BDFA00239A0002F1604247
:102BEC00013302F561424FF0FF31082BC2F880101F
:102BFC00C2F88011F1D1244B00241C635C639C63EC
:102C0C001C645C64FDF7F4FE20480121FDF7A0FF75
:102C1C0021461E48FDF79CFFF1200121FDF7A4FF82
:102C2C002146F120FDF7A0FF01200146FDF7A8FF8A
:102C3C0021460120FDF7A4FF15480121FDF7ACFF4B
:102C4C0021461348FDF7A8FF12480121FDF7B0FFFC
:102C5C0010482146FDF7ACFF63B64FF0FF3EB5467A
:102C6C002847042000F01AFA022000F017FA4FF45B
:102C7C00004000F01EFA23E700000108044550FE56
:102C8C00004000083E3F000800380240001060225F
:102C9C00FFC9FE36335907000748084A08B50849EA
:102CAC00121AFDF7CBF90748074A0021121AFDF753
:102CBC00CEF9FFF76DFB00BF0000002020000020C4
:102CCC00D43F000820000020480001202DE9F04FDF
:102CDC00DDE909AB0E469C4603783B490746C95CC7
:102CEC0001300D07F8D42B2B05D02D2B04D1074622
:102CFC004FF0FF3301E007460123397830290ED11C
:102D0C007978782905D132F0100103D102371022DD
:102D1C0007E00AB1082A04D10137082201E002B900
:102D2C000A2200200021B84617F8015BA5F13004F7
:102D3C00E4B2092C0DD9A5F14104192C02D8A5F146
:102D4C00370405E0A5F16104192C30D8A5F157041E
:102D5C00E4B294422BDA4FEAE27900FB09F502FB6C
:102D6C000155A0FB0201E4B2294400194FF0000503
:102D7C0041EB0501BCF1000FD5D0012B06D18245EA
:102D8C007BEB0104CFDA50465946CCE75C1CCAD128
:102D9C00DDE90B89444261EB4105444575EB0909BA
:102DAC00C1DADDE90B01404261EB4101BBE70EB139
:102DBC00C6F80080DD1700FB05F203FB0122A0FB27
:102DCC0003011144BDE8F08F4C1200082DE9F04FBF
:102DDC0091B01F9E0C46310691468046DDE91A23C0
:102DEC001E9D04D5CDE902234FF0000C1BE0002AF8
:102DFC0073F100071046194602DA504263EB4301A7
:102E0C00002A73F1000ACDE9020107DBB70708D4E9
:102E1C0016F0040C07D04FF0200C04E04FF02D0CF2
:102E2C0001E04FF02B0C16F04007089714BF704FC1
:102E3C00704FDDE902AB079700271C980137C117CB
:102E4C00CDE90401DDE904230AA93944099150466E
:102E5C005946CDF804C0FEF773FA07980999835CBC
:102E6C00504601F8013C5946DDE90423FEF768FAA7
:102E7C0082468B465AEA0B02DDF804C001D0162FAD
:102E8C00DBD116F0080239461DD01C9B082B02D052
:102E9C00102B0ED01CE0DDE902AB1DB95AEA0B0B6E
:102EAC0013D004E05AEA0B0B12D0BD4210DC7B1C91
:102EBC000FE0DDE902AB5AEA0B0B09D008982B4660
:102ECC0048B1582208E02B4606E02A46012303E0CD
:102EDC002B46002200E078221CF1000B1D98C7EB5A
:102EEC00030A18BF4FF0010BBB42A8BF1F46C01B03
:102EFC002AEAEA7ACBEB00000AB1022700E0174677
:102F0C00C71B16F0010027EAE77701D07F4205E0E6
:102F1C00F60603D5013504BFBA4407463D46002DDD
:102F2C000BDD2068013D461C4E453CBF202608F8B1
:102F3C000060206801302060F1E727EAE7703F1A53
:102F4C00BBF1000F08D02068451C4D4538BF08F870
:102F5C0000C02068013020608AB12068451C4D45B6
:102F6C003CBF302508F800502568681C02354D45DB
:102F7C00206038BF08F80020226801322260BAF1C4
:102F8C00000F0CD022680AF1FF3A501C48453CBF98
:102F9C00302008F80200226801322260EFE7DDE9F8
:102FAC0002AB5AEA0B0B10D17BB919460DE0236822
:102FBC0001395A1C4A4505D201F1280568462A5C9C
:102FCC0008F803202368013323600029EFD15FB197
:102FDC00236801375A1C4A453CBF202208F80320BD
:102FEC00236801332360F2E711B0BDE8F08F00BF16
:102FFC009A3F0008AB3F00081EF0040F0CBFEFF324
:10300C000880EFF30980FEF7C3BF7047032970B542
:10301C0005460C4606D98E083146FDF7FFFBB60077
:10302C003544A41B14B9FDF707FC70BD00231846EA
:10303C00EA5C0133A34242EA0020F9D1FDF7E8FB38
:10304C0070BD2DE9F0410733DE08079B4FF01208E5
:10305C0008FB02320731069F054602EBD10800241B
:10306C00BC4209D0122000FB048029463246FCF7F2
:10307C00E5FF01343544F3E7BDE8F08106235843FE
:10308C0001387FF4FDAF704710B504460020FDF702
:10309C000BFF20420CBF0020012010BD10B50446D0
:1030AC000020FDF701FF20EA04010020FDF7ECFEF3
:1030BC0010BD10B504460020FDF7F6FE40EA0401F1
:1030CC000020FDF7E1FE10BD1FB501A8FEF759F871
:1030DC000723029301A803230393FDF7B1FD684670
:1030EC00FEF755F869460020FDF7EEFD05B05DF8DA
:1030FC0004FB70B50646FEF79FFC8020FEF716FC1D
:10310C00A82420BA90FAA0F0C0B2FEF70FFC11254B
:10311C00705DFEF70BFC15F1FF35F9D20020FEF7C0
:10312C0005FC013C06F11206EBD12046FEF7FEFB36
:10313C00FEF766FC70BD38B500242546E0B2FEF7FC
:10314C0029FEA04001340543042CEDB2F6D12846EB
:10315C0038BD08B50D20FEF7D3FB0A20FEF7D0FBD7
:10316C0008BD10B5441E14F8010F10B1FEF7C8FBD2
:10317C00F9E710BD08B5FFF7F4FFFFF7EAFF08BD4C
:10318C001FB530238DF8043078238DF805300723D4
:10319C0099000F228A400240CA40092A01D83032D5
:1031AC0002E00F2A02D85732D2B200E0202201A945
:1031BC00CC1A13F1FF336272EAD2002308468DF861
:1031CC000E30FFF7CEFF04B010BD70B504460D46AF
:1031DC004FF4805001211646FDF7AEFCFEF7F2FDD0
:1031EC000520FEF7DDFEA920FEF7DAFEC307FAD4B0
:1031FC00FEF7BEFDFEF7E6FD0320FEF7D1FEC5F39C
:10320C000740FEF7CDFEC5F30720FEF7C9FEE8B276
:10321C00FEF7C6FE2644B44205D0A920FEF7C0FE38
:10322C0004F8010BF7E7FEF7A3FD4FF480500021E3
:10323C00FDF782FC70BD0000000000001F000000C4
:10324C003B0000005A0000007800000097000000CE
:10325C00B5000000D4000000F300000011010000D4
:10326C00300100004E010000000000080040000882
:10327C000080000800C000080000010800000208DF
:10328C000000040800000608863F00080008024001
:10329C00080000008B3F0008000002400400000002
:1032AC008E3F00080008024040000000953F0008D7
:1032BC00000002400200000000000240010000007B
:1032CC000000080010001800200028003000380012
:1032DC000000068301000000000000000000000058
:1032EC00068301000000000C0000000000000683B3
:1032FC0001000000000C00000000D878369B79C05B
:10330C00E3D90C8C67DB3C1BF8FD7EBFFDE0F7FBC3
:10331C001FC6EFFB7E1F98CD66B3CD60369B19C6DA
:10332C006C18660398FD66B3FD60309B19C66F1868
:10333C00660398FD66B3FD60309B19C36F18660376
:10334C00980D66B30D60369B19C360186603F8FDC3
:10335C007EBFFDECF79B19C36F187E03D878369BA4
:10336C0079CCE399998167183C03180000000000A0
:10337C0000008001000000001800000000000000A8
:10338C000000000000001800000000000000000019
:10339C0000000000000C000600000000600030007F
:1033AC000018000300000000C0001800003080016D
:1033BC000000000080010C000060C0000000000054
:1033CC000003060000C060000000000000060300BF
:1033DC000080310000000000008C010000001B0088
:1033EC000000000000D8000000000E0000000000EB
:1033FC000070000000000E000000000000700000D3
:10340C0000001B000000000000D80000008031000C
:10341C0000000000008C010000C0600000000000F3
:10342C00000603000060C00000000000000306005E
:10343C00003080010000000080010C000018000327
:10344C0000000000C0001800000C00060000000086
:10345C0060003000000000000000000000000000D0
:10346C000000000000000000000000000000000050
:10347C000000000000000000000000000000000040
:10348C000000000000000000000000000000000030
:10349C000000000000000000000000000000000020
:1034AC000000000000000000000000000000000010
:1034BC00000000000000000080FFFF010000000081
:1034CC0000000000FEFFFF7F00000000000000E095
:1034DC007F0000FE07000000000000FE01000080DD
:1034EC007F0000000000801F00000000F8010000B9
:1034FC000000F00100000000800F000000007C00C4
:10350C0000000000003E000000000F000000000062
:10351C0000F00000008003000000000000C001006B
:10352C0000E0000000000000000007000070000038
:10353C000000000000000E00001800000000000059
:10354C0000001800000C000000000000000030001B
:10355C0000060000000000000000600000030000F6
:10356C00000000000000C00080010000000000000E
:10357C0000008001C00000000000000000000003FB
:10358C006000000000000000000000063000000099
:10359C00000000000000000C100000000000000003
:1035AC00000000080000000000600000030018008C
:1035BC000000000000000060000003001800000084
:1035CC000000000000600000030018000000000074
:1035DC000000006000000300180000000000000064
:1035EC000060000003001800000000E003001F60F2
:1035FC00F800C30718C0070000F80FC07F60FE0377
:10360C00F31F18F01F00000C1860C06003061B307D
:10361C00181830000006303080E1010C0F60180CD7
:10362C0060000003601800E3001807C01806C00013
:10363C008001400C006200100380180380008001A0
:10364C00C00C006600300380190380018001C0FCAF
:10365C00FF670030038019FFFF018001C0FCFF638E
:10366C000030038019FFFF008001C00C00600030A7
:10367C000380190300008001C00C0060003003803F
:10368C00190300008001400C006200100380180335
:10369C0080008003601800C3001806C01806C00024
:1036AC00800730308081010C0C60180C6000800D9C
:1036BC001860C000030618303818300080F90FC0AD
:1036CC007F00FE03F01F70F01F0080E103001F005D
:1036DC00F800C00760C00700800100000000000077
:1036EC00000000000000800100000000000000004D
:1036FC00000000008001000000000000000000003D
:10370C00000080010000000000000000000000002C
:10371C0080010000000000000000000000004E6F5F
:10372C002048572056657273696F6E20696E204F62
:10373C0054500056335231007573622077616B65BB
:10374C00757020737570706F7274656400456E745B
:10375C006572696E67207374616E646279002069AA
:10376C0073206F7574736964652073797374656DF8
:10377C0020666C6173680048415244204641554CA8
:10378C005400446573636C656E20000A4669726D63
:10379C006C656E20000A5873756D20000A496E76B0
:1037AC00616C6964206669726D776172652064650D
:1037BC00736372697074696F6E2100436865636B23
:1037CC0073756D6D696E67206669726D7761726570
:1037DC002075706461746500496E76616C69642053
:1037EC006669726D776172652043524320696E2061
:1037FC0053504920666C6173682100657261736572
:10380C005F6F6C645F6669726D77617265004F6C97
:10381C006420576F726C64206669726D7761726593
:10382C002062617365006661696C656420746F2049
:10383C00657261736520736563746F7220007772B3
:10384C006974655F6E65775F6669726D77617265C5
:10385C00006661696C656420746F207772697465A9
:10386C00206164647265737320005765277265204C
:10387C006465616400436865636B73756D6D696E37
:10388C00672000206279746573004E657720576F4E
:10389C00726C64206669726D7761726520737973DE
:1038AC0074656D5F666C6173685F62617365004F10
:1038BC006C6420576F726C64206669726D776172EC
:1038CC00652073797374656D5F666C6173685F6294
:1038DC0061736500436865636B73756D202D20778C
:1038EC00616E746564200020676F7420004F7572E0
:1038FC0020696E7465726E616C20666C61736820F1
:10390C00636F6E74656E747320617265206261649E
:10391C002028636865636B73756D206661696C65DF
:10392C006429212054686973206973207265616C65
:10393C006C79206261642100FFFFFFFFFFFFFFFF36
:10394C00FFFFFFFF010000000000000000000080EE
:10395C0001000000000000000000008001000000D9
:10396C0000000000000000800100000000000000CA
:10397C00000000800100000000000000000000803A
:10398C00010000000000000000000080FFFFFFFFAE
:10399C00FFFFFFFFFFFFFFFF7C00FE00FF01C701E1
:1039AC00C701C701C701C701C701C701C701C701CB
:1039BC00C701C701C701FF01FE007C0038003C00B5
:1039CC003E003E003800380038003800380038001F
:1039DC0038003800380038003800FE00FE00FE00C9
:1039EC007C00FE00FF01C701C701C001C001E0005F
:1039FC00F00078003C001E000E000F000700FF01D5
:103A0C00FF01FF017C00FE00FF01C701C701C001DF
:103A1C00C001F8007800F800C001C001C001C70166
:103A2C00C701FF01FE007C00E000E000F000F000A8
:103A3C00F800F800F800FC00EC00EE00E600FF01D6
:103A4C00FF01FF01E000E000E000E000FF00FF00EC
:103A5C00FF000700070007007F00FF00FF01C70100
:103A6C00C001C001C701C701C701FF01FE007C00F6
:103A7C007C00FE00FF01C701C701070007007700AB
:103A8C00FF00FF01C701C701C701C701C701FF0143
:103A9C00FE007C00FF01FF01FF01E000E000700070
:103AAC007000700038003800380038001C001C0012
:103ABC001C001C001C001C007C00FE00FF01C70148
:103ACC00C701C701C701FE007C00FE00C701C7018A
:103ADC00C701C701C701FF01FE007C007C00FE008E
:103AEC00FF01C701C701C701C701C701FF01FE01E3
:103AFC00DC01C001C001C701C701FF01FE007C0051
:103B0C0000000000000000007C00FE00FF01C70167
:103B1C00C701F001FC01CE01C701C701E701FF019C
:103B2C00DF01CE010700070007000700E700F701DF
:103B3C00FF01CF01C701C701C701C701C701C701F9
:103B4C00CF01FF01F701E7000000000000000000BA
:103B5C007C00FE00FF01C701C7010700070007003A
:103B6C000700C701C701FF01FE007C00C001C001B6
:103B7C00C001C001CE01DF01FF01E701C701C70190
:103B8C00C701C701C701C701E701FF01DF01CE0172
:103B9C0000000000000000007C00FE00FF01C701D7
:103BAC00C701C701FF01FF010700C701C701FF01E2
:103BBC00FE007C00E000F000F8003800FE00FE0083
:103BCC00FE00380038003800380038003800380063
:103BDC0038003800380038005341442057415443D2
:103BEC00483A200052657365742052656769737496
:103BFC006572200042726F776E206F75742072654B
:103C0C00736574005374617274696E67204C53450C
:103C1C00206F7363696C6C61746F72004C53452038
:103C2C006F7363696C6C61746F7220646964206E6D
:103C3C006F74207374617274005553422077616BFA
:103C4C00657570006C656176696E67207374616E62
:103C5C0064627900205F5F5F5F5F5F202020205FE0
:103C6C005F0D0A2F5F20205F5F2F205F5F2F202FBB
:103C7C000D0A202F202F2020202F5F20205F5F2F68
:103C8C000D0A2F5F2F20202020202F5F2F0D0A00E0
:103C9C00426F6F746C6F61646572207665727369C4
:103CAC006F6E3A20004C617374206669726D776197
:103CBC00726520626F6F7420776173207374616218
:103CCC006C653B20636C65617220737472696B6503
:103CDC007300537475636B20627574746F6E20720D
:103CEC006567697374657220697320696E76616C9F
:103CFC0069642C20636C656172696E672E00427575
:103D0C0074746F6E2069642000697320737475631A
:103D1C006B2100427574746F6E207761732070751F
:103D2C0073686564206F6E20626F6F742E2042750D
:103D3C0074746F6E20636F756E7465723A200042F6
:103D4C006F6F7420626974733A2000486F6C642042
:103D5C00646F776E205550202B204241434B2066D8
:103D6C006F72203520736563732E20746F20666F1D
:103D7C007263652D626F6F742050524600466972F3
:103D8C006D7761726520697320657261736564007B
:103D9C00426F6F74696E67206E6F726D616C6C79B7
:103DAC00005761746368646F672063617573656441
:103DBC00206120726573657400536F66747761724D
:103DCC0065206661696C75726520636175736564E5
:103DDC00206120726573657400426F6F7420666198
:103DEC00696C65642C20737472696B6520330042B6
:103DFC006F6F74206661696C65642C2073747269D2
:103E0C006B65203200426F6F74206661696C65646B
:103E1C002C20737472696B652031004C6F6164697E
:103E2C006E67207265636F76657279206669726D54
:103E3C0077617265004661696C656420746F206CF3
:103E4C006F6164207265636F766572792066697242
:103E5C006D776172652C20737472696B65206F6E5F
:103E6C00652E2054727920616761696E2E0046615F
:103E7C00696C656420746F206C6F6164207265637B
:103E8C006F76657279206669726D776172652C2028
:103E9C00737472696B652074776F2E20547279205D
:103EAC00616761696E2E004661696C656420746F90
:103EBC00206C6F6164207265636F76657279206621
:103ECC0069726D776172652C20737472696B6520F1
:103EDC0074687265652E2053414420574154434801
:103EEC00004F75722070726576696F757320666904
:103EFC00726D77617265207570646174652066619E
:103F0C00696C65642C2061626F7274696E672075D0
:103F1C0070646174652E004E6577206669726D77EA
:103F2C0061726520697320617661696C61626C6590
:103F3C002100426F6F74696E67206669726D7761DC
:103F4C0072652040200072657475726E696E672010
:103F5C00746F207374616E64627900466F7263656E
:103F6C002D626F6F74696E67207265636F76657210
:103F7C0079206D6F64652E2E2E004261636B0055A7
:103F8C00700053656C65637400446F776E0030315C
:103F9C0032333435363738394142434445460030A4
:103FAC0031323334353637383961626364656600D3
:103FBC00286E756C6C2900000000000102030401DE
:083FCC000203040607080900C6
:103FD40000A0000002020000FFFFFFFF00C0040178
:103FE40000000000000000021000000007000000B4
:040000050800134C90
:00000001FF
